:100000000C9434000C9451000C9451000C94510049
:100010000C9451000C9451000C9451000C9451001C
:100020000C9451000C9451000C9451000C9451000C
:100030000C9451000C9451000C9451000C945100FC
:100040000C9451000C9451000C9451000C945100EC
:100050000C9451000C9451000C9451000C945100DC
:100060000C9451000C94510011241FBECFEFD8E026
:10007000DEBFCDBF11E0A0E0B1E0ECE8F2E002C0ED
:1000800005900D92A230B107D9F721E0A2E0B1E0CE
:1000900001C01D92A530B207E1F70E94A2000C94A6
:1000A00044010C94000080910401880F80930401A6
:1000B0009091030197FD1DC0990F9093030189272B
:1000C0002091020127FD21C0220F20930201829579
:1000D0008695869583709091000197FD1AC0292F0F
:1000E000220F9227982791FD2F5F20930001822FE6
:1000F000089521E0280F20930401990F90930301A4
:1001000089272091020127FFDFCF9F5F9093030192
:10011000DBCF2F5F20930201E2CF02C000000197E6
:100120000097E1F70895009761F028EE3DEF000099
:100130002150310921153105D1F701970097A9F711
:100140000895089583E084B98CEF8AB917B88CE0DC
:1001500085B980EEC82E90ECD92E20EAE22E30E848
:10016000F32E00E610E4D0E2C0E00E94530081705C
:10017000C81BC23008F44AC0289A0E9453008170FC
:10018000D81BD23008F44AC0299A0E9453008170CB
:10019000181B123008F44AC05A9A0E94530081700A
:1001A000081B023008F44AC05B9A0E945300817019
:1001B000F81A81E08F1508F04AC05C9A0E9453003B
:1001C0008170E81A81E08E1508F04AC05D9A0E949D
:1001D00053008170D81A81E08D1508F04AC05E9AEC
:1001E0000E9453008170C81A81E08C1508F04AC043
:1001F0005F9A80E197E2000001970097E1F70E9483
:1002000053008170C81BC23008F0B6CF28980E94F6
:1002100053008170D81BD23008F0B6CF29980E94C5
:1002200053008170181B123008F0B6CF5A980E9404
:1002300053008170081B023008F0B6CF5B980E9413
:1002400053008170F81A81E08F1508F4B6CF5C98DE
:100250000E9453008170E81A81E08E1508F4B6CF31
:100260005D980E9453008170D81A81E08D1508F4C2
:10027000B6CF5E980E9453008170C81A81E08C1539
:0C02800008F4B6CF5F98B5CFF894FFCF1C
:02028C0001006F
:00000001FF
